:020000000628D0
:04000C00D02882076F
:1000100080340834983410349834043480340434F0
:1000200072340434AA341034AA34043498340434B6
:100030008F3408345F3410345F340434653404344E
:100040008034043472340434803410348034043402
:100050007234043472340834723404345534023443
:100060005F340834653404345F3404347234083443
:1000700080341034BF340434AA3404349834043443
:1000800072341034803404348F340434983404349B
:10009000BF340434BF34103482075F341034553415
:1000A00004344C340834403408344034083439348F
:1000B0000834403408344C3408345F341034553438
:1000C00004344C3408344C340834553408345F3428
:1000D0000834553410345F341034553404344C34FF
:1000E0000834403408344034083439340834403457
:1000F00008344C3408345F341034553410344C34E4
:1001000008344C340834553408345F3410344834DF
:10011000083448340834393408343934083439342C
:10012000083440340834403408344C3408345F34E4
:100130000834553410345F341034553404344C349E
:1001400008344034083440340834393408344034F6
:1001500008344C3408345F341034553404344C348F
:1001600008344C34083455340834553408345F347A
:1001700020348207BF341034BF340434BF34083411
:10018000BF340434BF34083498340434AA340834F7
:10019000BF340434BF340834CA340834BF34103494
:1001A00007309F008316FD3085000F3086008130B8
:1001B000810083128601203084008001840A041F9C
:1001C000DD2837083A3EB700F92010215F217C2155
:1001D000C721013A031D2F2AC80A872287228722B6
:1001E0003708343A031DE6283608033A031DE6288B
:1001F000572A06080F39003A0319080000309B00FF
:100200009A0183161C1555309D00AA309D009C1440
:100210001C119C18092983120230B3004B210800DD
:10022000B001C70A47080339B4008722B42110304F
:10023000B30030080720B100B00A30080720B20030
:1002400030218601B00A3008443A0319B00106088B
:100250000F39003A031911290230B3004B2108006D
:10026000AE012E083206031908003308AD0031082C
:100270008514402185104021AD0B3729AE0A312964
:10028000AC000000000000000000000000000000C2
:10029000AC0B41290800B101B1090130B200302195
:1002A000B10B4D2987228722872287228722872226
:1002B00087228722080001080339B40008005B2167
:1002C0003708840003103608003A03197329013AED
:1002D00003197129033A03196F29B40DB40DB40D34
:1002E000B40DB40DB40D000834048000B60A361DF8
:1002F0000800B601B70A0800B8013A30B900390859
:1003000084000008C7003808003A03199329013A0D
:1003100003199129033A03198F29C70CC70CC70C7D
:10032000C70CC70CC70C47080339B400A9218722A2
:1003300087228722B80A3819A62938083606031DED
:100340007F2939083706031908007F29B801B90A3F
:100350009D29B421B1002030B2001030051E0130BB
:10036000B3003021860108003408003A0319BF2980
:10037000013A0319C129033A0319C329C5290616ED
:100380005F3486164C340617403486173334051113
:100390008515B8013A30B900390884000008C70053
:1003A0003808003A0319E029013A0319DE29033A13
:1003B0000319DC29C70CC70CC70CC70CC70CC70C2A
:1003C00047080339B400FA21003A0319003435080C
:1003D0003406031D0034B80A3819F72938083606E0
:1003E000031DCC293908370603190134CC29B8017B
:1003F000B90AEE29B5010730051E0330AE00FF3003
:10040000AD00FF30AC000618122A8618162A06190D
:100410001A2A86191E2AAC0B032AAD0B012AAE0B31
:10042000FF2900340616B5015F30222A86163514DE
:100430004C30222A0617B5144030222A861735146C
:10044000B5143330B1002030B2000330B300302196
:1004500006080F39003A031D272A860101340130AE
:10046000B3004B210130B3004B217C21872287222E
:10047000872200309B0083161C1483121A0848023E
:100480000318572AB0011030B30087223008B92072
:10049000B100B00A3008B920B2003021B00A3008EB
:1004A000163A031D452A872287228722DA28003040
:1004B0009B0048089A0083161C1555309D00AA30F1
:1004C0009D009C141C119C18632A8312B001C70A5A
:1004D00047080339B4008722B4210530B30030083F
:1004E0004C20B100B00A30084C20B2003021860107
:1004F000B00A30086C3A0319832A06080F39003A0B
:100500000319672ADA28872287228722DA28C3304C
:10051000AD00FF30AC00AC0B8B2AAD0B892A080074
:02400E00183F59
:00000001FF
